:020000040800F2
:1000000000090020E904000805150008091500088A
:100010005D1500080915000831150008EB040008FB
:10002000EB040008EB040008EB040008B5370008F7
:10003000EB040008EB040008EB040008593C00083E
:10004000EB040008EB040008EB040008EB040008D4
:10005000EB040008EB0400083D3A0008693A000888
:10006000953A0008C13A0008ED3A0008EB04000890
:10007000EB040008EB040008EB040008EB040008A4
:10008000EB040008EB040008EB04000875260008E8
:10009000E12600083527000889270008193B0008D9
:1000A000EB040008EB040008EB040008EB04000874
:1000B000EB040008EB040008EB040008EB04000864
:1000C000EB040008EB040008EB040008EB04000854
:1000D000EB040008EB040008452B0008592B00082E
:1000E000813B0008EB040008EB040008EB04000867
:1000F000EB040008EB040008EB040008EB04000824
:10010000EB040008EB040008EB040008EB04000813
:10011000EB040008EB040008EB040008EB04000803
:10012000EB040008EB040008EB040008EB040008F3
:10013000EB040008EB040008EB040008EB040008E3
:10014000EB040008EB040008EB040008EB040008D3
:10015000EB040008EB040008EB040008EB040008C3
:10016000EB040008EB040008EB040008EB040008B3
:10017000EB040008EB040008EB040008EB040008A3
:10018000EB040008EB040008EB040008EB04000893
:10019000EB040008EB040008EB040008EB04000883
:1001A000B114000800000000D0400B1CD1409C4658
:1001B000203AD34018435242634693401843704755
:1001C0009140031C90409C46203A93401943524270
:1001D0006346D3401943704753B94AB9002908BF51
:1001E00000281CBF4FF0FF314FF0FF3000F07AB90C
:1001F000ADF1080C6DE904CE00F006F8DDF804E07E
:10020000DDE9022304B070472DE9F0478C460D4626
:100210000446089E002B51D18A4217466DD9B2FA86
:1002200082FEBEF1000F0BD0CEF1200C01FA0EF5CC
:1002300020FA0CFC02FA0EF74CEA050C00FA0EF458
:100240004FEA174A250CBCFBFAF81FFA87F90AFB9C
:1002500018CC45EA0C4508FB09F3AB420AD9ED1965
:1002600008F1FF3280F02381AB4240F22081A8F1F7
:1002700002083D44ED1AA4B2B5FBFAF00AFB105592
:1002800044EA054400FB09F9A14509D9E41900F144
:10029000FF3380F00A81A14540F2078102383C44D7
:1002A000A4EB090440EA08400021002E61D024FAA2
:1002B0000EF4002334607360BDE8F0878B4207D9E9
:1002C000002E54D0002186E821000846BDE8F087C2
:1002D000B3FA83F1002940F08E80AB4202D3824210
:1002E00000F2FA80841A65EB03050120AC46002E6B
:1002F0003FD086E81010BDE8F08712B90127B7FBA0
:10030000F2F7B7FA87FEBEF1000F34D1EB1B3A0CBF
:100310001FFA87FC0121B3FBF2F8250C02FB18330E
:1003200045EA03450CFB08F3AB4207D9ED1908F188
:10033000FF3002D2AB4200F2D1808046ED1AA3B268
:10034000B5FBF2F002FB105543EA05440CFB00FC40
:10035000A44507D9E41900F1FF3302D2A44500F205
:10036000B8801846A4EB0C0440EA08409DE73146EB
:100370003046BDE8F087CEF1200405FA0EF307FA07
:100380000EF720FA04F83A0C25FA04F448EA0308B8
:10039000B4FBF2F14FEA184502FB11441FFA87FC47
:1003A00045EA044501FB0CF3AB4200FA0EF409D90F
:1003B000ED1901F1FF3080F08A80AB4240F2878076
:1003C00002393D44EB1A1FFA88F5B3FBF2F002FB49
:1003D000103345EA034500FB0CF3AB4207D9ED1996
:1003E00000F1FF386FD2AB426DD902383D44EB1AB1
:1003F00040EA01418FE7C1F1200722FA07F88B405C
:1004000005FA01F448EA030320FA07FE4FEA134C09
:10041000FD404EEA040EB5FBFCF94FEA1E440CFB0E
:1004200019551FFA83F844EA054509FB08F4AC4264
:1004300002FA01F200FA01FA08D9ED1809F1FF30C9
:1004400043D2AC4241D9A9F102091D442D1B1FFA28
:100450008EFEB5FBFCF00CFB10554EEA054400FB8C
:1004600008F8A04507D9E41800F1FF3529D2A045C6
:1004700027D902381C4440EA0940A4EB0804A0FB39
:1004800002894C45C6464D4615D312D056B1BAEB3B
:100490000E0364EB050404FA07F7CB401F43CC407E
:1004A000376074600021BDE8F0871846F8E6904692
:1004B000E0E6C245EAD2B8EB020E69EB030501386B
:1004C000E4E72846D7E7404691E78146BEE7014684
:1004D00078E702383C4445E7084608E7A8F10208F7
:1004E0003D442BE7704700BF02E000F000F8FEE754
:1004F00072B6394880F30888384880F3098838484C
:100500004EF60851CEF20001086040F20000CCF235
:1005100000004EF63471CEF200010860BFF34F8F39
:10052000BFF36F8F40F20000C0F2F0004EF688512A
:10053000CEF200010860BFF34F8FBFF36F8F4FF013
:100540000000E1EE100A4EF63C71CEF200010860A8
:10055000062080F31488BFF36F8F03F069F903F06E
:1005600095F94FF055301F491B4A91423CBF41F865
:10057000040BFAE71C49194A91423CBF41F8040BAD
:10058000FAE71A491A4A1B4B9A423EBF51F8040B2C
:1005900042F8040BF8E700201749184A91423CBF83
:1005A00041F8040BFAE703F047F903F0B1F9144CF2
:1005B000144DAC4203DA54F8041B8847F9E700F005
:1005C0003FF8114C114DAC4203DA54F8041B884734
:1005D000F9E703F02FB90000000900200011002006
:1005E0000000000800010020000900200844000865
:1005F000001100207411002078110020E026002056
:10060000A0010008A4010008A4010008A40100083A
:100610002DE9F04F2DED108AC1F80CD0C3689D462E
:10062000BDEC108ABDE8F08F002383F311882846C3
:10063000A047002002F0A2FE02F0CCFD00DFFEE7A2
:10064000394B6FF007022DE9F0416FF0670100248C
:100650001A7003225A709C70DC701C715C719C7162
:10066000DC711C7259729A72DC7203F04DF8074605
:1006700003F09AF80546D0BB2C4B9F4239D001338A
:100680009F4239D02A4B27F0FF029A4238D1F8B264
:1006900000F052FAA84642F2107400F08DFC00F00F
:1006A00051FA064680B38CBB464635B1214B9F427A
:1006B00003D003F071F800242646002003F02EF842
:1006C0004FF090431B6913F0200322D00EB100F0CD
:1006D00033F800F093FC00F027FE00F053FF0546CE
:1006E000CCB900F0E1FC012002F04EFEF8E78046B4
:1006F000D3E780460446D0E704464FF00108CCE734
:1007000080464FF47A74C8E70446CEE74FF47A7413
:10071000CBE71C46DDE700F035FF401BA042E0D9E7
:1007200000F00AF8D9E700BF78110020010007B0F7
:10073000000008B0263A09B010B51C4B1C4953F80C
:10074000042F013200D110BD8B42F8D1194C1A4B45
:1007500022689A4228D9194B9B6803F1006303F57C
:10076000D0439A4220D202F0EBFF02F0FDFF0020BE
:1007700000F0F4FD124B0220187000F02BFE114B1C
:10078000DA690022DA61D96999699A619B6972B65E
:100790000D4A0E4B13601B682268202181F31188DB
:1007A0009D4683F30888104710BD00BFFC67000812
:1007B0001C68000804680008FF6700087811002022
:1007C000841100200010024008ED00E000680008DD
:1007D00009490B6849F269009AB21B0C00FB02330D
:1007E000064A0B60136844F2506198B21B0C01FB7F
:1007F0000030106080B270470C11002008110020FA
:1008000010B500211022044600F0FEFD034B03CB7F
:10081000206061601868A06010BD00BFACF7FF1FCA
:10082000F0B51F4CBBB000F0ADFEA368C31AF92BA6
:1008300030D906AD2346A06028220021284601F0C9
:100840002FFC04F10E0000F0D7FD0023C6B2591DA5
:100850005F1CDBB2B3424FEAC10107DA0E33234417
:100860000822284601F01CFC3B46F0E701230393D5
:100870000823207B02930B4B0193C1F3CF0130235C
:10088000059100930146049503A3D3E9002306488C
:1008900001F0D6F93BB0F0BD78F6339F93CACD8D09
:1008A000E8210020F5210020C021002070B50D4670
:1008B00014461E4601F06AF950B9022E0ED1012CE1
:1008C0000CD112A3D3E90023C5E90023012070BD98
:1008D000052C14D003D8012C09D0002070BD282C81
:1008E00009D0302CF9D10BA3D3E90023ECE70BA3FB
:1008F000D3E90023E8E70BA3D3E90023E4E70BA344
:10090000D3E90023E0E700BFAFF30080401DA12042
:1009100026812A0B78F6339F93CACD8D9E6AC42117
:10092000818A46EE26417272DF25D7B7F017304A2A
:1009300039059E5638B504460D4603462022284602
:10094000002101F0ADFB22792346032A28BF0322B0
:1009500003F8042F28460222202101F0A1FB62792E
:100960002346072A28BF072203F8052F284603221B
:10097000222101F095FBA2792346072A28BF0722EE
:1009800003F8062F28460322252101F089FB28467B
:1009900004F108031022282101F082FB382038BD21
:1009A0002DE9F04FADF5017D21AE0EAD40F279128B
:1009B00080460F463046002100F026FD48220021E7
:1009C000284600F021FD00F0DDFD594B4FF47A720E
:1009D000B0FBF2F0186093E80700012385E80700F8
:1009E0002B740DF15A0000236B74FFF709FF0323EA
:1009F00085F82030F82385F8213007AB18464D499B
:100A000003F0E0F9192228643146284685F83C2095
:100A1000FFF790FF12AB044601460822304601F072
:100A20003FFB0822A1180DF14903304601F038FBC5
:100A30000DF14A03082204F11001304601F030FBA9
:100A400013AB202204F11801304601F029FB14AB4E
:100A5000402204F13801304601F022FB16AB082297
:100A600004F17801304601F01BFB0DF15903082217
:100A700004F18001304601F013FB04F1880A0DF106
:100A80005A0904F5847B4B465146082230460AF148
:100A9000080A01F005FBD34509F10109F3D11BABAD
:100AA00008225946304601F0FBFA04F588744FF0ED
:100AB000000995F834304B4510D84FF0000995F8EF
:100AC0003C304B4515D92B6C21464B44082230460F
:100AD00001F0E6FA083409F10109F0E7AB6B2146B1
:100AE0004B440822304601F0DBFA083409F10109D1
:100AF000DFE7E31DC3F3CF03F97E059300230496DC
:100B00000393BB7E0293193701230093019706A339
:100B1000D3E90023404601F093F80DF5017DBDE8CF
:100B2000F08F00BFAFF300809E6AC421818A46EE39
:100B300088110020E43E0008014B1870704700BF88
:100B4000B4110020F0B5314B1C7B85B034B1304B73
:100B50000E221A810024204605B0F0BD2D4A1068EF
:100B6000516802AB03C308230DEB03022A492B484B
:100B700003F0C6F8054630B9254B29480A221A81E8
:100B800000F0B6FCE6E70169B1F5663F06D9204BF7
:100B900024480B221A8100F0ABFCDCE7438BB3F551
:100BA0007E7F09D01A4A20480C2111814FF47E72B1
:100BB000194600F09DFCCEE71C4A024402F11003E6
:100BC0009942E4D310398E1A2046144900F0DEFC15
:100BD0003246074605F11801204600F0D7FCAB6805
:100BE0009F4202D1EB6898420AD0094B0D221A812C
:100BF00000903B46EA68A9680D4800F079FCA9E737
:100C00000C4800F075FC0124A5E700BFE821002096
:100C100088110020D43D0008DC970300006800081C
:100C2000DC3D0008E83D0008FA3D00080898FFF7A1
:100C3000183E0008413E00082DE9F04FADB006AF68
:100C400080460E4600F0A2FF044600286AD1337E9B
:100C5000022B18D1F38A012B15D100F093FC8146A9
:100C6000FFF7B6FD4FF4C873C14DB0FBF3F209F5C1
:100C7000167902FB1300F37E19FA80F028608BB915
:100C8000BC4B00221A709C37BD46BDE8F08F3B1D5F
:100C90001C440094002308224FEAC901304601F0A9
:100CA00063F84C46B38A013BA3425FFA84F90BD93F
:100CB00004F10109B9F1110FE9D1AF4BAF4A4FF47B
:100CC000A171AF4802F0EEFF07F11400FFF798FDA5
:100CD000224607F11401381D03F002F803460028EC
:100CE000CED1B9F1100F07D0A24B83F800902B683A
:100CF000A3F516732B60C6E707F19802014602F8C8
:100D0000950D30460092072201F02EF8F9787F29E0
:100D100004DD9C4B994A40F25911D2E7404600F05D
:100D200019FFB0E7F38A052B00F0348106D8012BB8
:100D3000A9D131464046FFF733FEA4E7282B3AD02D
:100D4000302BA0D1737E904C0133627BDBB2934297
:100D5000E94640F00581F27E237B9A4240F0008113
:100D600007F198034FF0000A23F884AD1022009396
:100D700051460123304600F0F7FFB58A023DADB27F
:100D8000EB1C23F003030A3323F00703ADEB030D41
:100D90000DF118085346991C9BB29D424FEAC101C0
:100DA0000AF1010A71DD4344009308220023304612
:100DB00000F0DAFFEEE7B38A013B9BB2C92B3FF6A6
:100DC00062AF714D71482022FF2100F01DFB2C7B8A
:100DD0004CBB05F10C030093082223462146304604
:100DE00000F0C2FFB38A04F10109013BE4B29C4266
:100DF0004FEAC90109DA0E342C440094002308227A
:100E0000304600F0B1FF4C46ECE700230022C5E974
:100E100000230023AB6085F8D730C5F8D8302B7B92
:100E20000BB9F37E2B73002407F114053B1D082238
:100E3000214628467C60BC60FC6001F031F93B7AB9
:100E400004F10109A3424FEAC90107D9FB6808224E
:100E50002344284601F024F94C46F0E7C1F3CF01C2
:100E60000023F07E059104950393B37E0293193617
:100E700028230146009301963BA3D3E90023404673
:100E800000F0DEFEFFF7CCFCFDE694F8D70000F0A2
:100E90006FFAD4F8D83082461BB994F8D70000F026
:100EA00077FAD4F8D8302B449A4504D294F8D70076
:100EB000013000F06DFA4FEA950B0026B1B25945AA
:100EC0001BDA94F8D73088007BB9D4E900231218D4
:100ED00043EBE073002B08BF202A06D22B4A58F8B8
:100EE000213042F821300136E8E7236808EB0001A1
:100EF0000122184400F090FAF5E7D4E90023D4F871
:100F0000D86094F8D700521943F100032E44C4E985
:100F10000023C4F8D86000F02BFA86420AD394F874
:100F2000D730013384F8D730D4F8D830A3EB0A0394
:100F3000C4F8D830FF2D0CDC08221449002020739F
:100F400000F06AFA00F036FAFFF7FCFD08B1FFF78F
:100F5000F3FB23680E4A9B0A013313810023A3602D
:100F6000CD4690E6AFF3008026417272DF25D7B7F9
:100F7000BC210020B9210020503E0008003F00089D
:100F8000A93E0008CB3E0008E82100209411002073
:100F900088110020BFF34F8F0549064BCA6802F441
:100FA000E0621343CB60BFF34F8F00BFFDE700BF8C
:100FB00000ED00E00400FA0508B54FF000530B4ABD
:100FC000196891420AD10A4A597D117009481B7D5E
:100FD0000373C92208490E3000F004FAE022002110
:100FE0004FF00050BDE8084000F00EBA9AAD44C57D
:100FF000B4110020E82100201600002030B5204C5C
:101000002049214885B00223637104230025ADF8EF
:1010100008300123ADF80C5007228DF80C308DF804
:101020000B301A4B4B608DF80A2001F023FE184B51
:10103000019500931749184B18484FF4805200F05F
:1010400053FD174B1978254611B1144800F082FD65
:1010500000F098FA0446FFF7BBFB4FF4C87304F5A1
:101060001674B0FBF3F202FB13000E4B14FA80F07F
:10107000186002F099FB08B10F232B8105B030BD39
:1010800088110020001100203823002003000600F2
:10109000AD080008B8110020390C0008C02100205C
:1010A000B4110020BC2100202DE9F04F94A7D7E90E
:1010B00000670FF25429D9E900898D4C93B0DFF80D
:1010C00050B2DFF850A2204600F006FE0CAD0790AB
:1010D00098B310220021284600F096F9079B197B4F
:1010E0004FF0000261F3030219468DF8302051F8E9
:1010F000040F49680EAA03C21B680D9A63F31C0211
:101100009DF830300D9243F020038DF830300023ED
:101110002A461946584601F0BDFD079030B92046D1
:1011200000F0DEFD079B8AF80030CCE79AF800302B
:10113000072B3EDC01338AF80030182200212846B4
:1011400000F062F9DFF8C8A1002319462A4650468C
:1011500001F0C8FD014680BB102208A800F054F938
:101160004FF09042536983F04003536100F00CFA52
:101170000B4612A9024611E903000DF1240E8EE878
:1011800003009DF83410C1F3030089064CBF0E998B
:10119000BDF838108DF82C0046BFC1F31C0141F09A
:1011A0000041C1F30A010891204608A900F0DEFFC2
:1011B000CAE7204600F094FDBFE7204600F0E6FCB9
:1011C000824600284AD1DFF850B100F0DBF9DBF8A5
:1011D0000030984242D300F0D5F90790FFF7F8FAB3
:1011E000079A8DF820A04FF4C87302F51672B0FB71
:1011F000F3F101FB130012FA80F0CBF80000DFF8E6
:101200001CB19BF8001011B901238DF8203028463D
:101210000791FFF7F5FA0799C1F1100A5FFA8AFA08
:10122000BAF1060F28BF4FF0060A524629440DF1C5
:10123000210000F0D7F80AF10103049308AB0393EF
:10124000182302932B4B01930123009332463B4614
:10125000204600F09DFC00238BF8003000F092F94E
:10126000254ADFF8BCA01368C31AB3F57A7F32D3DE
:10127000106000F089F902460B46204600F036FD6A
:10128000204600F083FC30B39AF80C30DFF894B0BD
:10129000002B14BF032302238BF8053000F072F9F2
:1012A0004FF47A732946B0FBF3F0CBF800005846B0
:1012B000FFF740FB182307300293104B0193C0F354
:1012C000CF0040F2551304900093039542464B46DD
:1012D000204600F05DFC9AF80C300BB1FFF7A0FA45
:1012E0009AF80C30002B7FF4EAAE13B0BDE8F08F13
:1012F000C0210020B8210020C8220020CC220020DC
:10130000401DA12026812A0BF1C6A7C1D068080F75
:1013100038230020CD220020BC210020B92100204C
:10132000E82100208811002070B502F0E3F8094C94
:10133000094E2070002530682378834208D902F0D6
:10134000D5F8336805440133B5F5D04F3360F2D397
:1013500070BD00BFFC220020D022002002F058B94E
:1013600000F10060920000F5D04002F0FDB80000EE
:10137000054B1A68054B1B789B1A834202D910440F
:1013800002F0B4B800207047D0220020FC220020D8
:1013900038B5074D04462868204402F0ADF828B956
:1013A00028682044BDE8384002F0B8B838BD00BF16
:1013B000D0220020064991F8243033B100230822BE
:1013C000086A81F82430FFF7CBBF0120704700BFC7
:1013D000D4220020022802BF4FF090434FF4800235
:1013E0009A61704710B50023934203D0CC5CC4547B
:1013F0000133F9E710BD000002460346981A13F9BD
:10140000011B0029FAD1704702440346934202D0DF
:1014100003F8011BFAE770472DE9F047234C94F8D5
:10142000243005468846174683BB2E46DFF87C905D
:10143000C7B394F824302BB92022FF2148462662F6
:10144000FFF7E2FF94F82400C0F10805BD4228BF71
:101450003D465FFA85FAAD0041462A4604EB80001E
:10146000FFF7C0FF94F82430A7EB0A079A445FFA0D
:101470008AFABAF1080F2E44A844FFB284F824A0D7
:10148000D6D1FFF797FF0028D2D108E0266A06EBF5
:101490008306B042CAD0FFF78DFF0028C5D10020D7
:1014A000BDE8F0870120BDE8F08700BFD42200200E
:1014B00070B50C4C1C26324600212046FFF7A4FFD5
:1014C000482323700125084B636065703246002174
:1014D000A019FFF799FF49232377044B657723620F
:1014E00070BD00BF0023002002040048060400482D
:1014F0000FB4002004B070470FB44FF0FF3004B0B9
:1015000070470000FEE7000000B59BB0EFF30981D3
:1015100068226846FFF766FFEFF30583034B9A6B7B
:101520009A6A9A6A9A6A9A6A9B6AFEE700ED00E0F4
:1015300000B59BB0EFF3098168226846FFF752FFC0
:10154000EFF30583044B9A6B9A6A9A6A9A6A9A6ACD
:101550009A6A9B6AFEE700BF00ED00E000B59BB011
:10156000EFF3098168226846FFF73CFFEFF305833C
:10157000034B5A6B9A6A9A6A9A6A9A6A9B6AFEE75E
:1015800000ED00E002F07CB802F056B830B5084D2E
:101590000A4491420BD011F8013B09245840013C08
:1015A000F7D040F300032B4083EA5000F7E730BD4B
:1015B0002083B8ED0246006848B103681360D38801
:1015C000118901339BB29942D38038BF1381704790
:1015D00070B588B00D460446202200216846FFF70A
:1015E00013FF20460495FFF7E5FF054658B16B460B
:1015F000044608AE1A4603CAB24220606160134630
:1016000004F10804F6D1284608B070BD2DE9F04178
:1016100030B9274B274A40F2C531274802F042FB38
:101620000B7C23B9254B234A40F2C631F5E7C66946
:1016300086B9C161BDE8F081002B29DA930CAB4279
:1016400029D1B44201D10C60F3E7C8F800100C6056
:10165000BDE8F0814B6823F06047BD0C4FEAD37EB4
:10166000C3F3807C15EA230538BF3D46B0463446B7
:101670006368BEEBD37F23F06042DDD1974203D194
:10168000C3F380739C450AD1974205E01C46EFE7FF
:10169000AA4206D013469D422CBF00230123002BF3
:1016A000CFD12368A046002BF0D12160BDE8F081A6
:1016B000D4410008C83F00088C420008AD42000831
:1016C00008B5034A034B044840F25E3102F0EAFADF
:1016D000A43F00084C4200088C42000808B503688B
:1016E0000B60C388016033B9044B054A05484FF4C9
:1016F000C76102F0D7FA013BC38008BD1C42000855
:10170000184000088C42000870B50C4600F10C052A
:10171000616831B9E38A61F30903E38200200021A3
:1017200070BD0E682846FFF7D9FF6660F0E700003D
:1017300008B5426832B10B4B0B4A0C4840F22F41BE
:1017400002F0B0FAC37DC3F38401013161F3860373
:10175000C375C38A62F30903C3821B0A62F3C7130A
:10176000C37508BD68420008D43F00088C420008D9
:101770002DE9F047089E32B91F4B204A204840F21D
:10178000395102F08FFA01F007054FEAD6082A44D2
:1017900006F0070600EBD1004FF47F49954201D1D6
:1017A000BDE8F08705F0070E06F0070AD645774634
:1017B00038BF5746C7F10807511BEC088F4228BFB6
:1017C0000F46045D08EBD60104FA0EF413F801C0CD
:1017D00029FA07FE24FA0AF45FFA8EFE8CEA040462
:1017E0004EFA0AFE04EA0E048CEA040C03F801C067
:1017F0003D443E44D2E700BFE8410008EC3F00080A
:101800008C4200082DE9F04106460F4600254FF6B0
:10181000FF7441F221082A4630463946FEF7C4FCDF
:10182000C0B284EA0024082314F4004F4FEA4404B1
:10183000A4B203F1FF3318BF84EA080413F0FF03D6
:10184000F2D10835402DE6D12046BDE8F0810000F8
:1018500010B50A4441F22104914200D110BD11F8A3
:10186000013B80EA0320082310F4004F4FEA4000B8
:1018700080B203F1FF3318BF604013F0FF03F3D1D0
:10188000EAE700002DE9F04F85B08A468DE80C00AC
:10189000BDF83C40814630B9494B4A4A40F26E316E
:1018A000494802F0FFF911F0604F04D0474B454A18
:1018B00040F26F31F4E7009B002B7ED024B10E9BE9
:1018C000002B7AD0072C28D809F10C00FFF772FE04
:1018D000054628B96FF00205284605B0BDE8F08F2F
:1018E00014220021FFF790FD22460E9905F1080011
:1018F000FFF778FD631C2B74009B1B782C4403F0CE
:101900001F0363F03F0323724AF000436B602946D4
:101910004846FFF77BFE0125DEE7019B1B0A4FF0DF
:101920000008029300F10C034FF0800B4646454639
:1019300003930398FFF73EFE07460028CAD01422FF
:101940000021FFF761FDB6BB9DF804303B729DF8A6
:1019500008307B7202220E9B711E1944B4420AD9D0
:10196000B8180132D2B211F801EF80F808E0013660
:10197000072AB6B2F2D1009B197801F01F01B442D8
:1019800008BF4FF0400BB81841EA48114BEA010379
:10199000037201324AF000437B603A74394648468C
:1019A000FFF734FE0135B4422DB288F001084FF044
:1019B000000BBED190E70022CDE76FF001058BE769
:1019C000D4410008B83F00088C420008F8410008E4
:1019D0002DE9F0471E46CB8A9146C3F30902062A39
:1019E00080460F4619D013460021B0B28DB25A1965
:1019F00092B2052A09D9A84210D8FA8A034463F39F
:101A00000902FA820120BDE8F087A842F3D93A44DE
:101A100019F8014094760131E8E70025FB8A7C68DB
:101A2000C3F30900821F1C23B2FBF3FA03FB1A2A3B
:101A30001FFA8AF27CB301212368002B39D1B31F2E
:101A400003441C20B3FBF0F301339BB299420CD248
:101A5000BAF1000F09D14046FFF7ACFD08B1C0F85C
:101A600000A0206008B304460022B6B24FF0000A7E
:101A7000B54230D2691E49441346E01801339BB287
:101A800011F801EF80F804E001351C2BADB214D041
:101A9000AE42F2D8ECE74046FFF78CFD044608B1B1
:101AA000002303607C60002CDED16FF00200BDE8F3
:101AB000F087013189B21C46BEE7AE42D8D9404614
:101AC000FFF778FD08B1C0F800A020600028ECD036
:101AD00004460022CCE7FB8AC3F30902164466F3EE
:101AE0000903FB828EE70000F8B50E4615461F4637
:101AF000044628B9144B154A15484F2102F0D2F874
:101B000024220021FFF780FC069B6360079B236271
:101B10006A094FF6FF739A424FF0000028BF1A4639
:101B2000A7602070A061E06197B204F10C058242C9
:101B300005D100232B6027826382A382F8BD2E602B
:101B4000013035462036F2E7D0410008443F000816
:101B50008C42000808B528B9084B094A7321094886
:101B600002F0A0F8037823B94BB2002B01DD01701D
:101B700008BD054B024A7D21F1E700BFD4410008B2
:101B8000503F00088C420008184100080078704758
:101B90002DE9F7430D9EBDF828900B9D9DF8304030
:101BA000BDF8388007461946104616B9B8F1000F3F
:101BB00043D11F2C41D83B78D3B9B8F1070F39D89E
:101BC00039F0030339D1424631464FF6FF70FFF733
:101BD0003FFE4FEA092920F0010009F44079400452
:101BE00049EA0464400C44EA40244FF6FF730DE0D8
:101BF00043EA0923B8F1070F43EA0464F5D9FFF774
:101C000001FE42463146FFF723FE03468DE84001C0
:101C10002A4621463846FFF735FE0DB9FFF750FD3D
:101C20002B780133DBB21F2B88BF00232B7003B04E
:101C3000BDE8F0836FF00300F9E76FF00100F6E70D
:101C40002DE9F7430E9F0B9D9DF83480BDF83C6055
:101C500081469DF8300007B9C6BB1F2836D899F8D1
:101C600000E0BEF1000F34D00C0244F080049DF877
:101C7000281044EAC83444EA014444EA0E04072E1A
:101C800044EA006415D919461046FFF7BBFD3246F9
:101C90003946FFF7DDFD0346019600972A462146A7
:101CA0004846FFF7EFFDB8F1010F0CD125B9FFF75A
:101CB00007FD4FF6FF73EFE72B780133DBB21F2BE5
:101CC00088BF00232B7003B0BDE8F0836FF00100E4
:101CD000F9E76FF00300F6E7C06900B10430704720
:101CE000C1690B68C3610C30FFF7F8BC2DE9F84FF0
:101CF000D0F818A0DFF86C80054616461F465446FB
:101D00004FF0000900F10C0B0CB9BDE8F88FD4E9D5
:101D10000223B21A67EB0303994508BF90451FD20F
:101D2000AB699C42214628460DD1FFF7EDFCAB691B
:101D30001B68AB6121465846FFF7D0FCAC692346CF
:101D4000A2461C46E0E7FFF7DFFC2368CAF8003034
:101D500021465846FFF7C2FC5446DAF80030EFE758
:101D60002368EDE780841E002DE9F04F8BB00D460F
:101D700014460793DDF850908246002800F06481F5
:101D8000B9F1000F00F06081531E3F2B00F25C811F
:101D9000012A03D1079B002B40F05681BAF814604A
:101DA000F6000023B5420893099380F053812B1964
:101DB0009E420AD2761B16F0FF0607D1AB4BAC4A07
:101DC00040F26751AB4801F06DFF2646DAF80C305F
:101DD00023B9DAF81030002B00F0A5802F2D31D870
:101DE000C5F1300846454FF000032CBF5FFA88F874
:101DF000B0460093294608AB4246DAF80800FFF7E0
:101E0000B7FCA6EB08074544FFB2BAF8143003F15B
:101E10000053063BDB000293DAF80C3005934FF0D9
:101E2000300B059B002B51D087B9DAF81000002841
:101E300061D0002F5FD0AB4550D98F4B8C4A40F218
:101E4000A651BFE737464FF00008DEE7029B23B9F3
:101E50008A4B874A4FF4B161B4E7029BE02B28BF5D
:101E6000E02306935B44AB4204931DD95B1B9F4266
:101E700026BFDBB203930397AB4504D97E4B7C4A64
:101E800040F291519EE70598CDF8008008ABA5EB94
:101E90000B01039A0430FFF76BFC039B9844FF1A75
:101EA0001D445FFA88F8FFB2049B9B4504D3744B32
:101EB0006F4A40F29B5185E7029B069ADDF810B00D
:101EC0009B1A0293059B1B680593AAE7029BBB42E2
:101ED000ABD26C4B664A40F2A15173E7CDF800805B
:101EE0003A46A5EB0B0108ABFFF742FCB8443D4472
:101EF0005FFA88F80027BAF81430B5EBC30F04D99D
:101F0000614B5B4A40F2B1515CE7B8F1400F04D934
:101F10005E4B574A40F2B25154E767B15C4B544AAA
:101F200040F2B3514EE70093324608AB2946DAF847
:101F30000800FFF71DFC731E3F2B35B201D8A642E7
:101F400004DD544B544A40F235213BE760070AD088
:101F50000AAB03EBD401624211F8083C02F007021D
:101F6000134101F8083C082C21D9102C21D9202C30
:101F70008CBF08230423079A002A6DD0B4EBC30F4B
:101F80006CD0082C04F1FF3215D89DF8203023FACC
:101F900002F2D10706D54FF0FF3202FA04F42343D0
:101FA0008DF820309DF8203089F800304EE0012374
:101FB000E1E70223DFE7102C11D8BDF8203023FA27
:101FC00002F2D20706D54FF0FF3202FA04F423439F
:101FD000ADF82030BDF82030A9F8003036E0202CD4
:101FE0000ED8089921FA02F2D30705D54FF0FF3336
:101FF00003FA04F40C430894089BC9F8003025E068
:10200000402C1CD0DDE9086730463946FEF7CCF895
:10201000002100F0010050EA01030BD0224601200C
:102020000021FEF7CDF8404261EB410106430F432A
:10203000CDE90867DDE90823C9E9002306E0174B6D
:10204000154A4FF42071BDE66FF0010528460BB02C
:10205000BDE8F08F1D46F9E7012CA3D0082CA1D9CB
:10206000102CB7D9202CE5D8C6E700BF24400008C3
:10207000FC3F00088C42000846400008334000083E
:102080006B40000893400008BA400008E840000890
:10209000004100081A4100087C3F00081841000870
:1020A00030B585B030B9244B244A40F2B1212448E0
:1020B00001F0F8FD23B9234B204A40F2B221F6E7A4
:1020C000402A04D9204B1D4A40F2B621EFE722B93D
:1020D0001D4B1A4A4FF42F71E9E70024012A02949C
:1020E000039417D11B788DF8083053070AD004AB3E
:1020F00003EBD203554213F8084C05F00705AC403A
:1021000003F8084C00910346002102A8FFF730FBBA
:1021100005B030BD082AE5D9102A03D81B88ADF8D0
:102120000830E2E7202A02D81B680293DDE7D3E9F2
:102130000045CDE90245D8E754410008903F00082A
:102140008C4200086F4100081841000870B50C4629
:1021500000F10C05E16819B9A1602161A18270BD8F
:102160000E682846FFF7BAFAE660F3E72DE9F04F6C
:10217000D1F8009091B0C9F3C01604460D46CDE9E0
:102180000223002E50D0C9F3C03BC9F30626B9F193
:10219000000F80F29F8119F0C04F40F09B812B7B94
:1021A000002B00F09781BBF1020F03D02278B242DE
:1021B00040F0938109F07F02BBF1020F059236D106
:1021C00019F07F0FC9F30F2A01D10AF0030A2B443B
:1021D0007606059A93F8038046EA0B4646EA82465D
:1021E0005FEAD81346EA0A06069300F09A800022B6
:1021F000002310A961E90823059B009367685B46EB
:1022000052462046B847002800F08880A7698FB959
:10221000314604F10C00FFF7DBF90746D0B96FF047
:10222000020011B0BDE8F08F4FF0020BAFE7C9F329
:10223000074ACCE73B699E420DD03F68002FF9D199
:10224000314604F10C00FFF7C3F907460028E6D039
:10225000A3693B60A761DDE90801FFF7D3FAB88203
:10226000F97D08F01F06C1F38401711A89B20FFAD3
:1022700081FED7E90223BEF1000FB8BF01F1200EA5
:10228000C9F30461B8BF0FFA8EFE079152EA030149
:1022900000F02F81DDE90201801A61EB03010246A3
:1022A0000B469F480021994208BF9042C0F021810F
:1022B000069B002B3FD0BEF1010F00F31A8118F0EE
:1022C000400F38D0DDE90223C7E902232022002194
:1022D0000DEB0200FFF798F8DDE90223CDE90823B2
:1022E0002B1D0A932B7BADF836A0013BDBB2ADF87A
:1022F00034309DF81C308DF83A309DF814308DF84C
:102300003B3020468DF838B08DF83960A36808A9B5
:1023100098473846FFF70CFA002082E76FF00B0071
:102320007FE7A76917B96FF00C007AE73B699E4217
:1023300096D03F68F6E7FB7DC8F34012B2EBD31F9F
:1023400040F0CE80C3F38403B34240F0CC800699C2
:102350002B7B4FEA981279B3D2073CD4032B40F27F
:10236000C580DDE90223C7E902232B7BAE1D033BB9
:10237000DBB23246394604F10C00FFF729FB002896
:1023800008DA39462046FFF7BFF93846FFF7D0F99B
:10239000032046E7AB883B832A7B033AD2B2B88A54
:1023A0003146FFF755FAFB7DB882DA43C2F3C0121B
:1023B00062F3C713FB75AFE76AB92E1D013BDBB2B1
:1023C0003246394604F10C00FFF702FB0028D8DB47
:1023D0002A7B013AE2E7FA8AC2F30902013B052AA5
:1023E000D9B250D8281D002399420AD907EB020E12
:1023F000013210F801CB8EF81AC00133062ADBB285
:10240000F2D1DDE902898B4207F11A02CDE9088990
:102410000A9238BF04337A680B9234BF5B190023E9
:102420000C93FB8AADF836A0C3F3090319449DF859
:102430001C308DF83A309DF814308DF83B30002375
:10244000ADF834108DF838B08DF839607B602A7B98
:10245000B88A013A291DFFF7FBF93B8BB88283420A
:1024600003D1A36808A92046984708A92046FFF78A
:102470006DFE3846FFF75CF9B88A3B8B984214BF73
:1024800011200020CDE6786810B34FF0060E0368E7
:102490009BB9A2EB0E021B2A13D80332024405F1AA
:1024A000040E1F309942ACD91EF801CB02F801CFBF
:1024B00001339042DBB2F5D1A3E70EF11C0E1846B2
:1024C000E5E7184B184A194840F2B31101F0EAFB4E
:1024D000034696E76FF00900A3E66FF00A00A0E656
:1024E0006FF00D009DE66FF00E009AE66FF00F00A2
:1024F00097E6FB7D68F386036FF3C713FB753946D8
:102500002046FFF701F9069B002B7FF4D8AEFB7D38
:10251000C3F38402013262F38603FB7503E700BF55
:1025200080841E0084410008683F00088C42000837
:102530002DE9F0414C4EB04240F081804B4CDFF829
:1025400030E1E56945F00075E561E469846AD4F835
:10255000007207EA0E0747F00107C4F80072D4F8CA
:10256000005205EA0E0545F0010545EA0121C4F8CF
:102570000012002A65D00021C4F81C120F46C4F8CE
:102580000412C4F80C12C4F8141204EBC105013192
:102590000E29C5F84072C5F84472F6D14FF0000E0E
:1025A0004FF0010C964510D1826AD2F80032B04249
:1025B00023F00103C2F8003253D12C4BDA6922F028
:1025C0000072DA61DB69BDE8F0819F781D8817F041
:1025D000010F18BFD4F804820CFA05F11CBF41EAC0
:1025E0000808C4F8048217F0020F1EBFD4F80C824A
:1025F00041EA0808C4F80C827F0742BFD4F814727D
:102600000F43C4F8147204EBC5055F68C5F8407247
:102610009F68C5F84472D4F81C522943C4F81C12B0
:102620000C330EF1010EBDE7846A0021C4F81C12C0
:10263000C4F80412C4F80C12C4F81412AEE7002A4D
:10264000F2D1836A0022C3F84022C3F84422C3F8BF
:102650000422C3F814220122C3F80C22C3F81C225E
:10266000A2E7BDE8F08100BF38230020001002403F
:102670000000FFFF184A916A08B58B688B6013F061
:10268000010105D013F00C0F14BF4FF4803101216C
:10269000D80506D513F4406F14BF41F4003141F062
:1026A0000201D80306D513F4402F14BF41F4802152
:1026B00041F00401D3690BB107489847202383F305
:1026C00011880021054800F087FE002383F311885C
:1026D000BDE8084001F07EB83823002040230020E8
:1026E00038B5124CA36ADD68AA0712D05A6922F0E5
:1026F00002025A61A36913B10121204698472023A1
:1027000083F3118800210A4800F066FE002383F35A
:102710001188EB0606D5A36A1021D960236A0BB194
:1027200002489847BDE8384001F054B838230020EB
:102730004823002038B5124CA36A1D69AA0712D09D
:102740005A6922F010025A61A36913B1022120468E
:102750009847202383F3118800210A4800F03CFEAB
:10276000002383F31188EB0606D5A36A10211961B3
:10277000236A0BB102489847BDE8384001F02AB8F7
:10278000382300204823002038B50F4CA36A5D6829
:102790005D602A070AD5032222701A6822F002021D
:1027A0001A60636A13B10021204698476B0706D56B
:1027B000A36A9969236A13B1090403489847BDE8DD
:1027C000384001F007B800BF3823002010B50F4C87
:1027D000204600F03DFA0E4BA3620B21132000F0BF
:1027E00017FA0B21142000F013FA0B21152000F02A
:1027F0000FFA0B21162000F00BFA002320461A4690
:102800000E21BDE81040FFF793BE00BF3823002023
:10281000006400400F4B984210B5044605D10E4BA2
:10282000DA6942F00072DA61DB69A36A01221A6098
:10283000A36A5A68D20707D5626851681268D961DD
:102840001A60064A5A6110BD0121082000F07CFC84
:10285000EEE700BF38230020001002405B87010034
:1028600003291AD8DFE801F0020A0F14836A9B6873
:1028700013F0E05F14BF012000207047836A98685E
:10288000C0F380607047836A9868C0F3C060704787
:10289000836A9868C0F3007070470020704700009A
:1028A00010B503291FD8DFE801F0021F2327816A32
:1028B0008B68C3F30163183301EB031310788106AF
:1028C0001ED55468C0F30011490041EAC40141F02B
:1028D000040100F00F00586090689860D268DA60D8
:1028E00041F00101196010BD836A03F5C073E5E78B
:1028F000836A03F5C873E1E7836A03F5D073DDE704
:102900009488C0F30011490041EA4451E1E7000016
:1029100001290CD003D3022910D000207047836A0C
:10292000DA68920701D1186903E001207047836AD1
:10293000D86810F0030018BF01207047836AF2E7DF
:1029400010B539B9836AD96889071BD11B699B0700
:1029500004D110BD012915D0022948D1816AD1F8CE
:10296000C031D1F8C401D1F8C8411461D1F8CC41CB
:10297000546120240C610C69A40717D14C6944F000
:10298000100412E0816AD1F8B031D1F8B401D1F865
:10299000B8411461D1F8BC4154612024CC60CC68AA
:1029A000A40703D14C6944F002044C6111795C081E
:1029B00064F304119C0864F34511117189064BBF3F
:1029C00091681189DB085B0D4CBF63F31C0163F355
:1029D0000A01137948BF916060F3030313714FEA52
:1029E00010234FEA104058BF11811370508010BD62
:1029F000002304491A465A50C8180833802B4260F5
:102A0000F9D17047642300200268436811430160D4
:102A100003B1184770470000024A136843F0C0032F
:102A20001360704700440040024A136843F0C0033B
:102A300013607047004800402DE9F047C66D3768C5
:102A4000F46934620546200719D014F0080F0CBF52
:102A500000218021E20748BF41F02001A30748BFC1
:102A600041F04001600748BF41F48071202383F3A7
:102A70001188281DFFF7C8FF002383F31188E205A2
:102A80000AD5202383F311884FF40071281DFFF726
:102A9000BBFF002383F311884FF020094FF0000A99
:102AA00014F0200831D13B0616D54FF0200905F16E
:102AB000380A200610D589F31188504600F04CFAE8
:102AC00000282FDA0821281DFFF79EFF27F080033A
:102AD0003360002383F3118879060DD562060BD588
:102AE000202383F31188EA6C2B6D9A4201D12B6C61
:102AF000F3B9002383F31188E30621D5AA6E136985
:102B0000F3B15069BDE8F047184789F31188B38CD9
:102B100095F864102846194000F0AAFA8AF3118843
:102B2000F469BDE780B2308588F31188F469C0E7A5
:102B30001021281D27F04007FFF766FF3760D8E710
:102B4000BDE8F08708B50348FFF776FFBDE8084009
:102B500000F040BEE423002008B50348FFF76CFFF7
:102B6000BDE8084000F036BE5024002037B51D4CAB
:102B70001D4D204600F070FA009404F1140000236B
:102B800020221A4900F032F92022009404F1380082
:102B9000174B184900F0ACF9174BE3652566174C45
:102BA0000C21262000F034F8204600F055FA04F1FC
:102BB0001400009400232022114900F017F904F1B9
:102BC000380000940F4B1049202200F091F90F4B70
:102BD000E3650C212720256603B0BDE8304000F0F6
:102BE00017B800BFE423002000512502BC240020B8
:102BF000192A0008FC240020004400405024002032
:102C0000DC240020292A00081C2500200048004060
:102C100000F1604300F01F02400903F56143090120
:102C20008000C9B200F1604083F8001300F56140F4
:102C300001239340C0F880310360704700F1604089
:102C4000090100F56D40C9B201767047FFF7BEBDBE
:102C500000F108020123037082600023C26000F1CA
:102C600010024360026142618361C3610362436297
:102C70007047000010B52023044683F31188022317
:102C800003704160FFF7C6FD03232370002383F325
:102C9000118810BD2DE9F0411F4604460D46164629
:102CA000202383F3118800F108082378042B0ED029
:102CB00029462046FFF7D4FD48B120463246294632
:102CC000FFF7EEFD002080F31188BDE8F081394662
:102CD000404600F065FB0028E7D0002383F311880D
:102CE000BDE8F0812DE9F0411F4604460D46164629
:102CF000202383F3118800F110082378042B0ED0D1
:102D000029462046FFF704FE48B1204632462946B0
:102D1000FFF716FE002080F31188BDE8F0813946E8
:102D2000404600F03DFB0028E7D0002383F31188E4
:102D3000BDE8F081F8B5154682680669AA420B46DF
:102D4000816938BF8568761AB542044607D21846AD
:102D50002A46FEF747FBA3692B44A3610DE011D976
:102D600032461846FEF73EFBAF1B3A46E168304458
:102D7000FEF738FBE2683A44A261A3685B1BA360DC
:102D80002846F8BD18462A46FEF72CFBE368E4E720
:102D900083682DE9F041044693421546266938BF01
:102DA00085684069361AB5420F4606D22A46FEF7B4
:102DB00019FB63692B4463610DE012D93246A5EB20
:102DC0000608FEF70FFB4246B919E068FEF70AFB5A
:102DD000E26842446261A3685B1BA3602846BDE8C9
:102DE000F0812A46FEF7FEFAE368E4E710B50A44EC
:102DF0000024C361029B006040608460C160816107
:102E000041610261036210BD08B582694369934262
:102E100001D1826882B98268013282605A1C4261A3
:102E20001970426903699A4201D3C3684361002162
:102E300000F0C6FA002008BD4FF0FF3008BD0000CA
:102E400070B5202304460E4683F31188A568A5B10A
:102E5000A368A269013BA360531CA3611578226992
:102E6000934224BFE368A361E3690BB1204698470E
:102E7000002383F31188284670BD3146204600F0B8
:102E80008FFA0028E2DA85F3118870BD2DE9F74F3B
:102E900005460F4690469A46D0F81C90202686F3A9
:102EA00011884FF0000B144664B12246394628467B
:102EB000FFF740FF034668B95146284600F070FA14
:102EC0000028F1D0002383F31188A8EB040003B09D
:102ED000BDE8F08FB9F1000F03D001902846C84734
:102EE000019B8BF31188E41A1F4486F31188DBE7FA
:102EF000C16081614161C3611144009B0060406019
:102F00008260016103627047F8B504460E461746B9
:102F1000202383F31188A568A5B1A368013BA360B2
:102F200063695A1C62611E70236962699A4224BFF8
:102F3000E3686361E3690BB120469847002080F3A2
:102F40001188F8BD3946204600F02AFA0028E2DA56
:102F500085F31188F8BD0000836942699A4210B573
:102F600001D182687AB98268013282605A1C82611A
:102F70001C7803699A4201D3C3688361002100F081
:102F80001FFA204610BD4FF0FF3010BD2DE9F74F5E
:102F900005460F4690469A46D0F81C90202686F3A8
:102FA00011884FF0000B144664B12246394628467A
:102FB000FFF7EEFE034668B95146284600F0F0F9E7
:102FC0000028F1D0002383F31188A8EB040003B09C
:102FD000BDE8F08FB9F1000F03D001902846C84733
:102FE000019B8BF31188E41A1F4486F31188DBE7F9
:102FF000026843681143016003B11847704700003D
:103000001430FFF743BF00004FF0FF331430FFF7D9
:103010003DBF00003830FFF7B9BF00004FF0FF336D
:103020003830FFF7B3BF00001430FFF709BF0000CE
:103030004FF0FF311430FFF703BF00003830FFF7C7
:1030400063BF00004FF0FF323830FFF75DBF000074
:1030500000207047FFF78ABD044B036000234360E4
:103060008360C36001230374704700BFC842000837
:1030700038B5C36904460D461BB904210844FFF75F
:10308000B7FF294604F11400FFF7BEFE002806DA58
:10309000201D4FF48061BDE83840FFF7A9BF38BD5F
:1030A000024B00221B605B609A6070473C25002049
:1030B000002303748268054B1B6899689142FBD218
:1030C0005A68036042601060586070473C250020D9
:1030D00008B5202383F31188037C032B05D0042B30
:1030E0000DD02BB983F3118808BD436900221A6003
:1030F0004FF0FF334361FFF7DBFF0023F2E790E877
:103100000C001A6002685360F2E7000000230374A9
:103110008268054B1B6899689142FBD85A68036026
:1031200042601060586070473C250020054B1969CB
:103130000874186802681A605360186101230374E8
:10314000FDF766BA3C25002030B54B1C87B005461C
:103150000A4C10D023690A4A01A800F059F9284600
:10316000FFF7E4FF049B13B101A800F06BF923699A
:10317000586907B030BDFFF7D9FFF8E73C250020BC
:10318000D130000838B50C4D41612B6981689A68CF
:103190009142044603D8BDE83840FFF789BF18467E
:1031A000FFF786FF01232C61014623742046BDE80A
:1031B0003840FDF72DBA00BF3C250020044B1A68AB
:1031C0001B6990689B68984294BF0020012070475B
:1031D0003C25002010B5084C236820691A6822603D
:1031E0005460012223611A74FFF790FF01462069A1
:1031F000BDE81040FDF70CBA3C25002008B5FFF7EC
:10320000DDFF18B1BDE80840FFF7E4BF08BD0000CE
:10321000FEE7000010B5174CFFF742FF00F0EAF898
:1032200080221549204600F06FF8012344F8180C5D
:103230000374124B124AD96821F4E0610904090CA5
:103240000A431049DA60CA6842F08072CA600E49C7
:103250000A6842F001020A601022DA77202283F81D
:103260002220002383F3118862B60848BDE810408D
:1032700000F06CB864250020F042000800ED00E08A
:103280000003FA05F0ED00E0001000E0F84200084D
:10329000F8B50F4C226A01322262224652F8141FFE
:1032A0009142154606D08B68013B8B6020266369EE
:1032B0009A6802B1F8BD1968DF68DA604D60616133
:1032C00082F311881869B84786F31188EFE700BFC9
:1032D0003C250020EFF3118020B9EFF30583202275
:1032E00082F311887047000010B558B9EFF30584D8
:1032F000C4F3080414B180F3118810BDFFF77EFFFA
:1033000084F3118810BD0000826002220274002242
:10331000427470478368A3F17C0243F80C2C026965
:1033200043F83C2C426943F8382C074A43F81C2CDC
:10333000C26843F8102C022203F8082C002203F87C
:10334000072CA3F1180070472906000810B52023A8
:1033500083F31188FFF7DEFF00210446FFF712FF19
:10336000002383F31188204610BD0000024B1B6927
:1033700058610F20FFF7DABE3C250020202383F39D
:103380001188FFF7F3BF000008B50146202383F33F
:1033900011880820FFF7D8FE002383F3118808BDA9
:1033A00049B1064B42681B6918605A60136043605C
:1033B0000420FFF7C9BE4FF0FF3070473C250020C6
:1033C0000368984206D01A68026050605961184636
:1033D000FFF76EBE7047000038B504460D46206802
:1033E000844200D138BD036823605C604561FFF70B
:1033F0005FFEF4E7054B03F114025A619A614FF046
:10340000FF32DA6100221A62704700BF3C250020BB
:1034100010B5C2600A4A036153699C68A1420CD886
:103420005C68036044602060586081609868411A5D
:1034300099604FF0FF33D36110BD091B1B68ECE7A7
:103440003C250020036881689A680A449A604268B3
:10345000136003685A600023C360024B4FF0FF32D1
:10346000DA6170473C25002000207047FEE700002D
:10347000704700004FF0FF3070470000BFF34F8FE0
:10348000024AD368DB07FCD4704700BF002002402B
:1034900008B5074B1B7853B9FFF7F0FF054B1A69C6
:1034A000120641BF044A5A6002F188325A6008BDD0
:1034B000C8260020002002402301674508B5054BBF
:1034C0001B7833B9FFF7DAFF034A136943F080032F
:1034D000136108BDC8260020002002407F289ABF43
:1034E00000F58030C0020020704700004FF40060FB
:1034F00070470000802070477F2808B50BD8FFF781
:10350000EDFF00F500630268013204D1043083420C
:10351000F9D1012008BD002008BD00007F2810B5AA
:1035200004461CD8FFF7AAFFFFF7B2FF0D4BF322AA
:10353000DA6002221A61FFF7D1FF58611A6942F07E
:1035400040021A61FFF79AFF4FF4006100F0F6F8AD
:10355000FFF7B4FF2046BDE81040FFF7CDBF0020C5
:1035600010BD00BF002002402DE9F84312F0010316
:10357000144606D0204B40F243221A600020BDE8DA
:10358000F88385181D4A954204D91B4A4FF41271DD
:103590001160F3E7FFF77CFFFFF770FFDFF86C8047
:1035A000451A4FF00109012C05EB01060F4604D81E
:1035B000FFF784FF0120BDE8F883C8F8109031F8C8
:1035C000023B3380FFF75AFF0020C8F81000338811
:1035D0003A889BB29A420DD0074B40F25F221A60A4
:1035E000074B1E60074B1C60074B1F60FFF766FF11
:1035F000BDE8F883023CD6E7C4260020FFFF03089D
:10360000B8260020C0260020BC2600200020024052
:10361000084908B50B7828B153B9FFF739FF0123E2
:103620000B7008BD23B1BDE808400870FFF746BF26
:1036300008BD00BFC826002038B5FFF74BFE0D4B74
:103640000D4A1C6A11684FF47A7303FB04F38B4232
:103650000A49D1E9004504D2003445F10105C1E928
:103660000045E41845F100051360FFF73DFE2046D4
:10367000294638BD3C250020CC260020D02600203D
:1036800008B5FFF7D9FF4FF47A720023FCF7A4FDC9
:1036900008BD00BF10B50244064B0439D2B29042B7
:1036A00000D110BD441C00B253F8200041F8040FB3
:1036B000E0B2F4E750280040104B30B51C6A2404F7
:1036C00007D41C6A44F440741C621C6A44F400442D
:1036D0001C620B4C236843F4807323600244094B43
:1036E0000439D2B2904200D130BD441C00B251F82E
:1036F000045F43F82050E0B2F4E700BF001002403E
:10370000007000405028004007B5012201A90020A8
:10371000FFF7C0FF019803B05DF804FB13B5044642
:10372000FFF7F2FFA04206D002A9012241F8044DA2
:103730000020FFF7C1FF02B010BD0000704700007D
:10374000074B45F255521A6002225A6040F6FF724A
:103750009A604CF6CC421A60024B01221A707047F4
:1037600000300040D9260020034B1B781BB1034BCF
:103770004AF6AA221A607047D9260020003000407D
:10378000034B1B689B0042BF024B01221A7070471B
:1037900024100240D8260020024B4FF080721A609D
:1037A000704700BF24100240014B1878704700BFDB
:1037B000D8260020064A536823F001035360EFF334
:1037C0000983683383F30988002383F311887047E2
:1037D00030EF00E010B5202383F31188104B5B68B5
:1037E00013F4006318D0F1EE103AEFF309844FF0B0
:1037F000807344F84C3C0B4BDB6844F8083CA4F164
:10380000680383F30988FFF7D9FC18B1064B44F825
:10381000503C10BD054BFAE783F3118810BD00BF83
:1038200000ED00E030EF00E0390600083C0600083B
:1038300070470000FEE70000084A094B09498B4227
:1038400004D3094A0021934205D3704752F8040F6C
:1038500043F8040BF3E743F8041BF4E7784400084B
:10386000E0260020E0260020E02600204B68436090
:103870008B688360CB68C3600B6943614B690362EB
:103880008B6943620B6803607047000008B5194BF1
:103890009A6A42F4FC029A629A6A22F4FC029A62E0
:1038A0009A6A5A6942F4FC025A61134A5B691146EA
:1038B0004FF09040FFF7DAFF104802F11C01FFF7CC
:1038C000D5FF0F4802F13801FFF7D0FF0D4802F194
:1038D0005401FFF7CBFF0C4802F17001FFF7C6FF60
:1038E0000A4802F18C01FFF7C1FFBDE8084000F073
:1038F00065B800BF001002401843000800040048EB
:1039000000080048000C004800100048001400485F
:1039100008B500F08FF9FFF77DFCBDE80840FFF720
:103920002FBF00007047000010B5214CA26A62F45E
:10393000FC02A262A26A02F4FC02A2624FF0FF3112
:10394000A26A226921612269002222612069E0685D
:10395000E160E168E260E168E169164841F08051A8
:10396000E161E169016841F480710160216A01F45B
:103970004071B1F5407F1EBF4FF480332362226255
:10398000236A1B0407D4236A43F440732362236A27
:1039900043F40043236200F02DF9A369064A43F083
:1039A0000103A361A369136843F02003136010BDF2
:1039B0000010024000700040000001401C4B1A68DB
:1039C00042F001021A601A689007FCD55A6822F08A
:1039D00003025A605A6812F00C02FBD1196801F018
:1039E000F90119605A601A6842F480321A601A6844
:1039F0009103FCD50F4A5A604FF40452DA62302228
:103A00001A631A6842F080721A601A689201FCD533
:103A1000094A122111605A6842F002025A605A683B
:103A200002F00C02082AFAD11A6B1A63704700BF21
:103A3000001002400024050000200240084A08B59A
:103A4000536911680B4003F00103536123B1054A28
:103A500013680BB150689847BDE80840FFF7BABE3D
:103A60000004014064230020084A08B55369116826
:103A70000B4003F00203536123B1054A93680BB175
:103A8000D0689847BDE80840FFF7A4BE0004014095
:103A900064230020084A08B5536911680B4003F0FD
:103AA0000403536123B1054A13690BB15069984768
:103AB000BDE80840FFF78EBE0004014064230020EB
:103AC000084A08B5536911680B4003F008035361B5
:103AD00023B1054A93690BB1D0699847BDE8084006
:103AE000FFF778BE0004014064230020084A08B5AF
:103AF000536911680B4003F01003536123B1054A69
:103B0000136A0BB1506A9847BDE80840FFF762BEE0
:103B10000004014064230020174B10B55C691A684B
:103B2000144004F478725A61A30604D5134A936AC8
:103B30000BB1D06A9847600604D5104A136B0BB1DD
:103B4000506B9847210604D50C4A936B0BB1D06B90
:103B50009847E20504D5094A136C0BB1506C98479D
:103B6000A30504D5054A936C0BB1D06C9847BDE80A
:103B70001040FFF72FBE00BF000401406423002067
:103B80001A4B10B55C691A68144004F47C425A61FF
:103B9000620504D5164A136D0BB1506D9847230585
:103BA00004D5134A936D0BB1D06D9847E00404D54A
:103BB0000F4A136E0BB1506E9847A10404D50C4AFE
:103BC000936E0BB1D06E9847620404D5084A136F08
:103BD0000BB1506F9847230404D5054A936F0BB17E
:103BE000D06F9847BDE81040FFF7F4BD00040140D6
:103BF00064230020062108B50846FFF709F80621CE
:103C00000720FFF705F806210820FFF701F8062135
:103C10000920FEF7FDFF06210A20FEF7F9FF062125
:103C20001720FEF7F5FF06212820BDE80840FEF723
:103C3000EFBF000008B5FFF777FEFEF7D9FEFFF7EC
:103C400005F8FFF707FAFFF76DFEBDE8084000F042
:103C500001B8000000F00EB808B5202383F31188E6
:103C6000FFF716FB002383F31188BDE80840FFF738
:103C7000B1BD0000054B064A5A6000229A60072237
:103C80001A6008210B20FEF7D9BF00BF10E000E04A
:103C90003F19010008B5062000F078F80120FFF771
:103CA000E5FB00001FB51C46094B1B680546D8689C
:103CB00052B1084B02928DE80A0022462B46064973
:103CC000FDF71AFCFFF7E6FF044B1A46F2E700BFC8
:103CD00010110020C0430008CD4300084F3E0008EB
:103CE00010B501390244904201D1002010BD10F8F6
:103CF000013B11F8014FA342F5D0181B10BD000085
:103D00002DE9F8430746884691461E468BB10D467D
:103D1000A8EB0500B54207EB000402D20020BDE885
:103D2000F883324649462046FFF7DAFF18B1013DD5
:103D3000EEE7BDE8F8832046BDE8F8831F2938B5D3
:103D400004460D4604D9162303604FF0FF3038BDFA
:103D5000426C12B152F821304BB9204600F030F8D5
:103D60002A4601462046BDE8384000F017B8012B2E
:103D70000AD0591C03D116230360012038BD00244A
:103D800042F8254028469847002038BD024B01469E
:103D90001868FFF7D3BF00BF1011002038B5074CDB
:103DA00000230546084611462360FFF763FB431CCA
:103DB00002D1236803B12B6038BD00BFDC26002090
:103DC000FFF752BB034611F8012B03F8012B002A21
:103DD000F9D1704740A2E4F1646891064E6F20610A
:103DE0007070207369670A00426164206677206CF6
:103DF000656E6774682025750A0042616420626FF1
:103E00006172645F69642025752073686F756C64E6
:103E10002062652025750A0042616420617070206F
:103E2000435243203078253038783A30782530387E
:103E300078203078253038783A3078253038780A4C
:103E400000476F6F64206669726D776172650A0062
:103E500072656365697665645F756E697175655FC6
:103E600069645F6C656E203C2055415643414E5F4E
:103E700050524F544F434F4C5F44594E414D49436C
:103E80005F4E4F44455F49445F414C4C4F43415462
:103E9000494F4E5F554E495155455F49445F4D412D
:103EA000585F4C454E475448002E2E2F2E2E2F542F
:103EB0006F6F6C732F41505F426F6F746C6F6164F2
:103EC00065722F63616E2E63707000616C6C6F633E
:103ED000617465645F6E6F64655F6964203C3D205A
:103EE000313237006F72672E6172647570696C6F62
:103EF000742E48697465634D6F73616963000000D7
:103F0000766F69642068616E646C655F616C6C6F6C
:103F1000636174696F6E5F726573706F6E7365282D
:103F200043616E617264496E7374616E63652A2CBD
:103F30002043616E61726452785472616E7366657B
:103F4000722A290063616E617264496E69740000AF
:103F500063616E6172645365744C6F63616C4E6F24
:103F6000646549440000000063616E6172644861E9
:103F70006E646C6552784672616D650063616E6156
:103F800072644465636F64655363616C61720000C1
:103F900063616E617264456E636F64655363616CE7
:103FA00061720000696E6372656D656E7454726152
:103FB0006E73666572494400656E7175657565540A
:103FC000784672616D6573007075736854785175C9
:103FD0006575650070726570617265466F724E65D9
:103FE00078745472616E736665720000636F7079E5
:103FF0004269744172726179000000006465736304
:1040000061747465725472616E7366657250617921
:104010006C6F61640000000066726565426C6F63DE
:104020006B0000006269745F6C656E677468203EA7
:1040300020300072656D61696E696E675F626974D8
:1040400073203E203000696E7075745F6269745F22
:104050006F6666736574203E3D20626C6F636B5FB4
:104060006269745F6F666673657400626C6F636B20
:104070005F656E645F6269745F6F66667365742006
:104080003E20626C6F636B5F6269745F6F6666731C
:1040900065740072656D61696E696E675F626974EF
:1040A0005F6C656E677468203C3D2072656D616968
:1040B0006E696E675F6269747300696E7075745FB4
:1040C0006269745F6F6666736574203C3D2074722C
:1040D000616E736665722D3E7061796C6F61645FAD
:1040E0006C656E202A2038006F75747075745F627D
:1040F00069745F6F6666736574203C3D20363400DA
:1041000072656D61696E696E675F6269745F6C6527
:104110006E677468203D3D20300028726573756CB1
:1041200074203E2030292026262028726573756C65
:1041300074203C3D203634292026262028726573C1
:10414000756C74203C3D206269745F6C656E6774A9
:104150006829000064657374696E6174696F6E200C
:10416000213D202828766F6964202A29302900768D
:10417000616C756520213D202828766F6964202AAE
:10418000293029006F66667365745F7769746869A2
:104190006E5F626C6F636B203C2028333255202D9C
:1041A000205F5F6275696C74696E5F6F66667365C8
:1041B000746F66202843616E61726442756666653D
:1041C00072426C6F636B2C2064617461292900005A
:1041D0006F75745F696E7320213D202828766F69A2
:1041E00064202A29302900007372635F6C656E2099
:1041F0003E203055000000002863616E5F69642036
:104200002620307831464646464646465529203DCA
:104210003D2063616E5F696400000000616C6C6F3B
:104220006361746F722D3E73746174697374696332
:10423000732E63757272656E745F75736167655F07
:10424000626C6F636B73203E203000007472616E8D
:10425000736665725F696420213D202828766F6946
:1042600064202A293029000073746174652D3E6230
:1042700075666665725F626C6F636B73203D3D208F
:104280002828766F6964202A293029002E2E2F2EA7
:104290002E2F6D6F64756C65732F6C696263616E30
:1042A0006172642F63616E6172642E63006974656C
:1042B0006D2D3E6672616D652E646174615F6C6523
:1042C0006E203E2030000000000000001D3000087D
:1042D0000930000845300008313000083D30000842
:1042E000293000081530000801300008513000085E
:1042F0006D61696E000000001043000880250020F9
:10430000B826002001000000113200080000000063
:1043100069646C6500000000A0100000000000004F
:10432000FAAAAAAA50040000BFFF0000007700000C
:10433000000000001410AA0000000000AAAAFAAAB7
:1043400004005000FBFF000000000000997700000F
:104350000000000000000000AAAAAAAA00000000B5
:10436000FFFF00000000000000000000000000004F
:1043700000000000AAAAAAAA00000000FFFF000097
:10438000000000000000000000000000000000002D
:10439000AAAAAAAA00000000FFFF00000000000077
:1043A000000000000000000000000000AAAAAAAA65
:1043B00000000000FFFF00000000000000000000FF
:1043C0002C2066756E6374696F6E3A20006173739A
:1043D000657274696F6E2022257322206661696C94
:1043E00065643A2066696C6520222573222C206C56
:1043F000696E65202564257325730A000CBEFF7F56
:104400000100000000000000640000000000000047
:10441000FE2A0100D2040000141100200000000058
:10442000000000000000000000000000000000008C
:10443000000000000000000000000000000000007C
:10444000000000000000000000000000000000006C
:10445000000000000000000000000000000000005C
:10446000000000000000000000000000000000004C
:0C44700000000000000000000000000040
:00000001FF
